:020000040800F2
:1000000000040020A10200089110000895100008CB
:10001000E910000895100008BD100008A3020008B0
:10002000A3020008A3020008A30200081529000883
:10003000A3020008A3020008A3020008A30200080C
:10004000A3020008A3020008A3020008A3020008FC
:10005000A3020008A3020008653E0008913E0008C4
:10006000BD3E0008E93E0008153F0008A302000855
:10007000A3020008A3020008A3020008A3020008CC
:10008000A3020008A3020008A3020008A3020008BC
:10009000A3020008A3020008A3020008413F0008D1
:1000A000A3020008A3020008A3020008A30200089C
:1000B000A3020008A3020008A3020008A30200088C
:1000C000A3020008A3020008A3020008A30200087C
:1000D000A3020008A3020008A3020008A30200086C
:1000E000A93F0008A3020008A3020008A302000819
:1000F000A3020008A3020008A3020008A30200084C
:10010000A3020008A3020008D53A0008A3020008D1
:10011000A3020008A3020008A3020008A30200082B
:10012000A3020008A3020008A3020008A30200081B
:10013000A3020008A3020008A3020008A30200080B
:10014000A3020008A3020008A3020008A3020008FB
:10015000A3020008A3020008A3020008A3020008EB
:10016000A3020008A3020008A3020008A3020008DB
:10017000A30200084D340008A3020008A3020008EF
:10018000A3020008A302000879110008A3020008D6
:10019000A3020008A3020008A3020008A3020008AB
:1001A000A3020008A3020008A3020008A30200089B
:1001B000A3020008A3020008A3020008A30200088B
:1001C000A3020008A3020008A3020008A30200087B
:1001D000A302000839340008A3020008A3020008A3
:1001E000A3020008A3020008A3020008A30200085B
:1001F000A3020008A3020008A3020008A30200084B
:10020000A3020008A3020008A3020008A30200083A
:10021000A3020008A3020008A3020008A30200082A
:10022000A3020008A3020008A3020008A30200081A
:10023000A3020008A3020008A3020008A30200080A
:10024000A3020008A3020008A3020008A3020008FA
:10025000A3020008A3020008A3020008A3020008EA
:10026000A3020008A3020008A3020008A3020008DA
:10027000A3020008A3020008A3020008A3020008CA
:10028000A3020008A3020008A3020008A3020008BA
:10029000A3020008A3020008A3020008A3020008AA
:1002A00002E000F000F8FEE772B6394880F30888F3
:1002B000384880F3098838484EF60851CEF20001DC
:1002C000086040F20000CCF200004EF63471CEF22D
:1002D00000010860BFF34F8FBFF36F8F40F2000043
:1002E000C0F2F0004EF68851CEF200010860BFF374
:1002F0004F8FBFF36F8F4FF00000E1EE100A4EF604
:100300003C71CEF200010860062080F31488BFF330
:100310006F8F02F03DFB03F05BFB4FF055301F4940
:100320001B4A91423CBF41F8040BFAE71C49194AA9
:1003300091423CBF41F8040BFAE71A491A4A1B4B99
:100340009A423EBF51F8040B42F8040BF8E7002034
:100350001749184A91423CBF41F8040BFAE702F0F2
:100360005BFB03F0A9FB144C144DAC4203DA54F8C8
:10037000041B8847F9E700F03FF8114C114DAC42DF
:1003800003DA54F8041B8847F9E702F043BB000086
:1003900000040020002400200000000800000020CD
:1003A0000004002000440008002400204424002011
:1003B0004824002060350020A0020008A0020008A8
:1003C000A0020008A00200082DE9F04F2DED108AD0
:1003D000C1F80CD0D0F80CD0BDEC108ABDE8F08F7D
:1003E000002383F311882846A047002001F0F0FE87
:1003F00001F0A0FE00DFFEE738B5204C6FF00803E7
:10040000002523700323A57063701E23E5702571FA
:100410006571A571E57125726572A372E57200F0D0
:1004200047FD20B10E2325726572A372E57202F0BA
:1004300033FA044602F068FA0546D0B9104B9C42E4
:1004400019D001339C4241F2883412BF0546002482
:100450000125002002F02AFA0DB100F0B7F800F0F3
:10046000BDFD00F07DFC204600F070F900F0AEF814
:10047000F9E70024EDE70446EBE700BF482400203D
:10048000010007B008B500F0E9FBA0F120035842D5
:10049000584108BD054B07B51B88022101A8ADF8DE
:1004A000043000F047FC03B05DF804FBB0400008E6
:1004B000064991F8243033B100230822086A81F8F4
:1004C000243000F071BC0120704700BF6824002078
:1004D0002DE9F84F234C05468846174694F82430FA
:1004E0008BBB2E46DFF87C90002F38D094F824A0E8
:1004F000BAF1000F05D12022FF214846266200F004
:100500005BFDCAF10805414604EB8A00BD4228BFE5
:100510003D465FFA85FBAD00A7EB0B072A462E444C
:1005200000F022FD94F82430A844FFB29B445FFA07
:100530008BFBBBF1080F84F824B0D5D1FFF7B8FFCF
:100540000028D1D108E0266A06EB8306B042C9D064
:10055000FFF7AEFF0028C4D10020BDE8F88F0120CE
:10056000BDE8F88F6824002010B5202383F311889C
:100570001248C3680BB101F0B1FE0023104A4FF4DA
:100580007A710E4801F06EFE002383F311880D4C42
:10059000236813B12368013B2360636813B1636868
:1005A000013B6360084B1B7833B9636823B90220B1
:1005B00000F0C6FC3223636010BD00BF542400204D
:1005C000690500089825002090240020554B5649C5
:1005D0002DE9F04153F8042F013201D1BDE8F0813B
:1005E0008B42F7D1514C524B22689A4240F298808C
:1005F000504B9B6803F1006303F500339A4280F08F
:100600008F80002000F0C8FB02204B4B187000F0D8
:1006100087FC4A4BD3F8E8200022C3F8E820D3F83F
:100620001011C3F81021D3F81011D3F8EC10C3F84F
:10063000EC20D3F81411C3F81421D3F81411D3F813
:10064000F010C3F8F020D3F81811C3F81821D3F82C
:100650001811D3F8801041F00061C3F88010D3F86E
:10066000801021F00061C3F88010D3F88010D3F817
:10067000801041F00071C3F88010D3F8801021F091
:100680000071C3F88010D3F8803072B62C4B2D491E
:100690000B601D682468BFF34F8FBFF36F8F2A4B29
:1006A000C3F88420BFF34F8F5A6922F480325A6115
:1006B000BFF34F8FD3F8802043F6E07EC2F3C90624
:1006C000C2F34E32B707520102EA0E0838463146ED
:1006D000013948EA000C00F14040B1F1FF3FC3F896
:1006E00074C2F5D1203A12F1200FEDD1BFF34F8F34
:1006F000BFF36F8FBFF34F8FBFF36F8F5A6922F431
:1007000000325A610022C3F85022BFF34F8FBFF36B
:100710006F8F202383F31188AD4685F30888204727
:10072000BDE8F081FCFF01081C000208040002087B
:10073000FFFF0108482400209024002000440258B4
:100740000000020808ED00E000ED00E02DE9F04FA8
:1007500099B0B34C2022FF21019010A8A66800F0A8
:100760002BFCB04AA3461378A3B90121AE481170FF
:10077000C360202383F31188C3680BB101F0AEFD81
:100780000023AA4A4FF47A71A74801F06BFD0023B9
:1007900083F31188019B13B1A54B019A1A600023C2
:1007A000A44AA349019F99461C461D4698461370CA
:1007B0004B600292012000F0B3FB002F00F0128288
:1007C0009B4B1B68002B40F00D8219B0BDE8F08FE9
:1007D0000220FFF757FE002840F0FB81019BB9F192
:1007E000000F08BF1F46944B1B8802210BA8ADF8D1
:1007F0002C3000F09FFADDE74FF47A7000F02EFA0B
:10080000031E0393EADB0220FFF73CFE824600282A
:10081000E4D0039B581E042800F2DD81DFE800F0DD
:10082000030E1114170018A80523042140F8343DC5
:1008300000F080FA54464FF0000856E00421784852
:10084000F6E704217D48F3E704217D48F0E71C2406
:100850002046043400F0A2FA04210B900BA800F00B
:1008600069FA2C2CF4D1E5E7002DB7D0002CB5D0D7
:100870000220FFF707FE0546002800F0AF810120A7
:100880006C4C00F089FA4FF000090220207000F053
:1008900047FB5FFA89FA504600F08EFA074658B1D6
:1008A000504609F1010900F097FA0028F1D12C46D1
:1008B000A9460027634B97E701233E460220237099
:1008C00000F01CFBDBF808309E4206D2304600F0F8
:1008D00065FA0130EBD10436F4E70026029BA94605
:1008E0002C461E703746524B5E6000F06DFB15B112
:1008F000002C18BF0027FFF7CDFD5BE7002D3FF46C
:100900006DAF002C3FF46AAF0220029B187000F01C
:1009100007FB322000F0A2F9B0F1000AC0F25E81BC
:100920001AF0030540F05A8106EB0A03DBF80820B1
:10093000934200F25381BAF5807F00F24F81554512
:100940000DDA4FF47A7000F089F90490049B002BC3
:10095000C0F24481049B3C4AAB540135EFE7C82008
:10096000FFF790FD0546002800F038811F2E11D8B2
:10097000C6F1200410AB26F0030033495445184457
:1009800028BF5446224600F0EFFA2246FF212E48A7
:1009900000F012FB4FEAAA0A2B4930465FFA8AF2AE
:1009A000FFF796FD0446002800F01A8106EB8A0640
:1009B00005469AE70220FFF765FD00283FF40EAFD9
:1009C000FFF776FD00283FF409AF4FF0000A5346C9
:1009D000DBF8082092451CD2BAF11F0F12D8109AEA
:1009E00001320FD02AF0030218A90A4452F8202C31
:1009F0000B92184604220BA90AF1040A00F088FBA6
:100A00000346E5E75046039300F0C8F9039B0B90BB
:100A1000EFE718A8042140F84C3D00F08BF964E79B
:100A20004824002094250020542400206905000853
:100A30009825002090240020B24000084C2400207B
:100A400050240020B44000089424002018A800235B
:100A5000642140F8343D00F039F900287FF4BEAE3F
:100A60000220FFF70FFD00283FF4B8AE0B9800F00E
:100A7000C5F918AB43F8480D04211846CDE718A86E
:100A80000023642140F8343D00F020F900287FF471
:100A9000A5AE0220FFF7F6FC00283FF49FAE0B98AE
:100AA00000F0AEF918AB43F8440DE5E70220FFF77C
:100AB000E9FC00283FF492AE00F0A8F918AB43F827
:100AC000400DD9E70220FFF7DDFC00283FF486AE99
:100AD0000BA9142000F0A0F9824618A8042140F8C0
:100AE0003CAD00F027F951460BA896E7322000F004
:100AF000B5F8B0F1000AFFF671AE1AF0030F7FF4FB
:100B00006DAE0AEB0803DBF8082093423FF666AEB1
:100B10000220FFF7B7FC00283FF460AE2AF0030A7A
:100B2000C244D0453FF4E1AE404608F1040800F06D
:100B300035F904210A900AA800F0FCF8F1E74FF417
:100B40007A70FFF79FFC00283FF448AEFFF7B0FC37
:100B500000283FF4AFAE109B01330CD0082210A93F
:100B60000020FFF7B5FC00283FF4A4AE2022FF21AF
:100B700010A800F021FAFFF78DFC374801F02EFB9A
:100B800023E6002D3FF42AAE002C3FF427AE18A830
:100B90000023642140F8343D00F098F88246002894
:100BA0007FF41CAE0220FFF76DFC00283FF416AE68
:100BB0000390FFF76FFC41F28830574601F00EFBBF
:100BC0000B9800F045FA00F0FFF9039B1C461D4608
:100BD000F0E5054689E64FF00008FFE52546FDE50E
:100BE0002C4667E6002000F039F80490049B002BA7
:100BF000FFF6E3AD012000F081F9049B213B122BAD
:100C00003FF6D8AD01A252F823F000BFD10700088B
:100C1000F907000869080008B5070008B5070008CB
:100C2000B5070008FD080008ED0A0008B50900082E
:100C30004D0A00087F0A0008AD0A0008B507000841
:100C4000C50A0008B50700083F0B0008EB080008BC
:100C5000B5070008830B0008A08601002DE9F347C3
:100C60004FF47A75002402AE154F4543DFF85880E3
:100C700006F8014D97F900305FFA84F95A1C01D04B
:100C8000A34212D158F82400012231460368D3F858
:100C900020A02B46D047012807D10A4B9DF807001A
:100CA00083F8009002B0BDE8F0870134022CE1D156
:100CB0004FF4FA7001F092FA4FF0FF30F2E700BF04
:100CC00000240020BC250020C84000082DE9F04782
:100CD0004FF47A7506460024134F4D43DFF85080D9
:100CE00097F900305FFA84F95A1C01D0A34210D161
:100CF00058F82400042231460368D3F820A02B467C
:100D0000D047042805D1094B002083F80090BDE8A6
:100D1000F0870134022CE3D14FF4FA7001F05EFA4F
:100D20004FF0FF30BDE8F08700240020BC250020F4
:100D3000C8400008074B30B41A78074B53F82240DC
:100D40000A46014623682046DD69044BAC4630BCA8
:100D5000604700BFBC250020C8400008A0860100F5
:100D6000F8B50A4C00250A4E01F07EFC094F2070B0
:100D700030682378834207D901F072FC3368054458
:100D80000133BD423360F3D9F8BD00BFBD2500205B
:100D9000A0250020FFFF010001F032BD00F100603E
:100DA00000F500300068704700F10060920000F527
:100DB000003001F0B5BC0000054B1A68054B1B78EC
:100DC0009B1A834202D9104401F04ABC00207047AC
:100DD000A0250020BD25002038B5074D0446286811
:100DE000204401F043FC28B928682044BDE838407D
:100DF00001F04EBC38BD00BFA02500200020704788
:100E0000014BC058704700BF00E8F11F014B186844
:100E1000704700BF0010005C234BF0B5234C1B68EB
:100E20002788C3F30B0665681B0C94F90820BE42A3
:100E300028D0A789BE4206D101220C2505FB024419
:100E4000656894F9082041F20104A3421CD041F2E4
:100E50000304A3421AD042F20104A34218D042F282
:100E60000304A34208BF5622441E013D0B460C4416
:100E7000A34217D215F9016F581C5EB1034600F862
:100E8000016CF5E70022D8E75A22EDE75922EBE79B
:100E90005822E9E72C2584421D7001D9981C5A700C
:100EA000401AF0BD1846FBE70010005C0424002047
:100EB000104B41F201015B888B429AB211D041F292
:100EC00003018B420FD042F201039A420DD042F24D
:100ED00003039A420BD10323074A02EB8303D8781A
:100EE00070470023F8E70123F6E70223F4E7002028
:100EF000704700BF0010005CB8400008022804D111
:100F00004FF48032044B9A6170470128FCD14FF4B2
:100F10008002024BF7E700BF0004025800000258AD
:100F2000022803D10122044B9A6170470128FCD1A9
:100F30004022024BF8E700BF0004025800000258AC
:100F4000022805D1064A536983F0010353617047B3
:100F50000128FCD1034A536983F04003F6E700BF40
:100F60000004025800000258002310B5934203D039
:100F7000CC5CC4540133F9E710BD000030B5441E09
:100F800014F9010F0B4658B193F900500131854215
:100F900006D11AB993F90020801A30BD013AEFE763
:100FA000002AF7D1104630BD02460346981A13F9BD
:100FB000011B0029FAD1704702440346934202D034
:100FC00003F8011BFAE77047024B1A78024B1A70BC
:100FD000704700BFBC2500200024002038B5164C07
:100FE000164D204600F02CFC2946204600F054FC0B
:100FF0002D681348D5F89020D2F8043843F0020346
:10100000C2F8043801F0EAF80E49284600F054FD11
:10101000D5F890200C48D2F804380C49A04223F0AF
:101020000203C2F804384FF4E1330B6003D0BDE88B
:10103000384000F063BB38BDEC2A0020A84100080E
:1010400040420F00C841000840260020A42500208F
:1010500038B50B4B05461A780A4B53F822400A4B19
:101060009C420CD0094B002118221846FFF7A4FF20
:10107000056001462046BDE8384000F03FBB38BD62
:10108000BC250020C8400008EC2A0020A425002030
:10109000FEE7000000B59BB0EFF3098168226846C7
:1010A000FFF762FFEFF30583034B9A6B9A6A9A6A24
:1010B0009A6A9A6A9B6AFEE700ED00E000B59BB071
:1010C000EFF3098168226846FFF74EFFEFF30583CF
:1010D000044B9A6B9A6A9A6A9A6A9A6A9A6A9B6AA3
:1010E000FEE700BF00ED00E000B59BB0EFF3098123
:1010F00068226846FFF738FFEFF30583034B5A6B0E
:101100009A6A9A6A9A6A9A6A9B6AFEE700ED00E018
:1011100030B50A44074D91420BD011F8013B092428
:101120005840013CF7D040F300032B4083EA5000C5
:10113000F7E730BD2083B8ED002304491A465A5022
:10114000C81808334260802BF9D17047C0250020B1
:10115000024A136843F0C0031360704700780040F0
:10116000044B5A6810439A6858600AB1181D10471A
:10117000704700BF402600202DE9F84F414EF56D25
:101180002F68EC6921072C6219D014F0080F0CBFEE
:1011900000208020E20748BF40F02000A3074FF066
:1011A000200348BF40F04000610748BF40F4807012
:1011B00083F31188FFF7D4FF002383F31188E2053E
:1011C00009D5202383F311884FF40070FFF7C8FF7F
:1011D000002383F311884FF02009DFF8A8A04FF017
:1011E000000B14F0200832D13B0615D54FF0200932
:1011F000DFF894A020060FD589F31188504600F03F
:10120000F1F9002830DA0820FFF7AAFF27F0800361
:101210002B60002383F3118879060DD562060BD568
:10122000202383F31188F26C336D9A4201D1336C21
:1012300003BB002383F31188E30604D5B26E136960
:101240000BB150699847BDE8F84F01F073BB89F3C3
:101250001188AB8C504696F86410194000F05CFA87
:101260008BF31188EC69BCE780B2288588F311887C
:10127000EC69BFE727F040071020FFF771FF2F60F0
:10128000D7E700BF402600207826002013B5104C79
:10129000204600F027FA04F11400009400234FF4D4
:1012A00000720C4900F0E8F804F1380000944FF4A3
:1012B0000072094B094900F061F9094B0C215220D9
:1012C000E365084B236602B0BDE8104000F05EB84D
:1012D00040260020AC26002051110008AC28002038
:1012E0000078004000E1F505254B002908BF1946AC
:1012F000037C012B816630B511D1224B98420ED16F
:10130000214BD3F8E82042F08042C3F8E820D3F81C
:10131000102142F08042C3F81021D3F810310A683E
:10132000036EC46D03EB5203B3FBF2F34A6815047A
:1013300042BF23F0070503F0070343EA4503E360D8
:101340008B6843F040036360CB68510543F00103B1
:10135000A36042F4967343F0010323604FF0FF3320
:10136000236205D512F0102205D0B2F1805F04D0BF
:1013700080F8643030BD7F23FAE73F23F8E700BFF1
:10138000EC400008402600200044025800F1604371
:1013900000F01F020901400903F56143C9B2800052
:1013A00083F80013012300F16040934000F5614091
:1013B000C0F8803103607047F8B51546826804466E
:1013C0000B46AA4200D28568A1692669761AB54201
:1013D00007D218462A46FFF7C7FDA3692B44A3612D
:1013E0000DE011D9AF1B32461846FFF7BDFD3A4656
:1013F000E1683044FFF7B8FDE2683A44A261A368AF
:1014000028465B1BA360F8BD18462A46FFF7ACFDD3
:10141000E368E4E7836893422DE9F04104460F4610
:10142000154600D2856860692669361AB54207D22A
:101430002A463946FFF798FD63692B4463610EE045
:1014400013D9A5EB060832463946FFF78DFD424613
:10145000B919E068FFF788FDE26842446261A36859
:1014600028465B1BA360BDE8F0812A463946FFF79A
:101470007BFDE368E2E7000010B50A440024C36185
:10148000029B006040608460C160816141610261D3
:10149000036210BD08B582694369934201D1826835
:1014A00082B98268013282605A1C426119704269B5
:1014B00003699A4201D3C3684361002100F0AAFE88
:1014C000002008BD4FF0FF3008BD000070B520239C
:1014D00004460E4683F31188A568A5B1A368A269E6
:1014E000013BA360531CA36115782269934224BF7A
:1014F000E368A361E3690BB120469847002383F3B7
:101500001188284670BD3146204600F073FE002841
:10151000E2DA85F3118870BD2DE9F74F05460F46D5
:1015200090469A46D0F81C90202686F311884FF0FA
:10153000000B144664B1224639462846FFF73CFFAB
:10154000034668B95146284600F054FE0028F1D001
:10155000002383F31188A8EB040003B0BDE8F08FEB
:10156000B9F1000F03D001902846C847019B8BF3C7
:101570001188E41A1F4486F31188DBE7C16081619A
:1015800041611144C361009B006040608260016161
:1015900003627047F8B504460E461746202383F3CE
:1015A0001188A568A5B1A368013BA36063695A1CB3
:1015B00062611E70236962699A4224BFE3686361B5
:1015C000E3690BB120469847002080F31188F8BDED
:1015D0003946204600F00EFE0028E2DA85F3118835
:1015E000F8BD0000836942699A4210B501D1826852
:1015F0007AB98268013282605A1C82611C78036960
:101600009A4201D3C3688361002100F003FE2046A3
:1016100010BD4FF0FF3010BD2DE9F74F05460F46C6
:1016200090469A46D0F81C90202686F311884FF0F9
:10163000000B144664B1224639462846FFF7EAFEFD
:10164000034668B95146284600F0D4FD0028F1D081
:10165000002383F31188A8EB040003B0BDE8F08FEA
:10166000B9F1000F03D001902846C847019B8BF3C6
:101670001188E41A1F4486F31188DBE70268436887
:101680001143016003B11847704700001430FFF7A1
:1016900043BF00004FF0FF331430FFF73DBF0000A1
:1016A0003830FFF7B9BF00004FF0FF333830FFF795
:1016B000B3BF00001430FFF709BF00004FF0FF3147
:1016C0001430FFF703BF00003830FFF763BF00009E
:1016D0004FF0FF323830FFF75DBF00000020704749
:1016E000FFF7D4BD044B0360002343608360C360F5
:1016F00001230374704700BF0441000810B5202384
:10170000044683F31188FFF7EFFD022323740023BF
:1017100083F3118810BD000038B5C36904460D4637
:101720001BB904210844FFF7A9FF294604F114005E
:10173000FFF7B0FE002806DA201D4FF48061BDE8F7
:101740003840FFF79BBF38BD026843681143016012
:1017500003B118477047000013B5446BD4F89434B4
:101760001A681178042915D1217C022912D119791E
:10177000012312898B4013420CD101A904F14C00C2
:1017800001F096FFD4F894440246019B2179206829
:1017900000F0EAF902B010BD143001F019BF0000EA
:1017A0004FF0FF33143001F013BF00004C3001F054
:1017B000EBBF00004FF0FF334C3001F0E5BF0000FD
:1017C000143001F0E7BE00004FF0FF31143001F09B
:1017D000E1BE00004C3001F0B7BF00004FF0FF3217
:1017E0004C3001F0B1BF0000D0F8942438B5136834
:1017F00005461978042901D0012038BD017C022951
:10180000FAD1127901205C8990400440F4D105F1AD
:10181000140001F079FE02460028EDD0D5F894546A
:101820004FF480732868697900F08CF9204638BD40
:10183000406BFFF7D9BF00000020704770470000E1
:101840007FB5124B01250226044603600023057470
:1018500000F18402436029468360C3600C4B029010
:10186000143001934FF48073009601F029FE094B68
:1018700004F523722946019304F14C004FF4807360
:101880000294009601F0F0FE04B070BD2C410008F7
:1018900031180008591700080A68202383F31188BB
:1018A0000B790B3342F823004B79133342F82300B2
:1018B0008B7913B10B3342F823000223C0F8941440
:1018C0000374002383F311887047000038B5037F49
:1018D000044613B190F85430ABB90125201D022104
:1018E000FFF732FF04F1140025776FF0010100F0DB
:1018F0009DFC84F8545004F14C006FF00101BDE8E8
:10190000384000F093BC38BD10B5012104460430C6
:10191000FFF71AFF0023237784F8543010BD00002E
:1019200038B504460025143001F0E2FD04F14C0006
:10193000257701F0B1FE201D84F854500121FFF7F6
:1019400003FF2046BDE83840FFF74EBF90F88030D7
:1019500003F06003202B19D190F88120212A0AD0AE
:10196000222A4FF000030ED0202A0FD1084A4267E6
:101970000722826704E0064B43670723836700233F
:10198000C3670120704743678367F9E7002070470A
:101990001C240020D0F8943437B51A680446117816
:1019A00004291AD1017C022917D11979012312893E
:1019B0008B40134211D100F14C05284601F02CFF59
:1019C00058B101A9284601F073FED4F894440246A8
:1019D000019B2179206800F0C7F803B030BD0000FA
:1019E00001F10B03F7B550F8234005460E46F4B15C
:1019F000202383F3118805EB8607201D08214C3432
:101A0000FFF7A2FEFB685B691B6813B1204601F07B
:101A10005DFE01A9204601F04BFE024648B1019B44
:101A20003146284600F0A0F8002383F3118803B064
:101A3000F0BDFB685A691268002AF5D01B8A013B89
:101A40001340F1D105F18002EAE70000133138B507
:101A500050F82140DCB1202383F31188D4F894247A
:101A60001368527903EB8203DB689B695D6845B1BB
:101A700004216018FFF768FE294604F1140001F004
:101A80004DFD2046FFF7B0FE002383F3118838BDDB
:101A90007047000001F048B8012300F1300200F166
:101AA000500103700023436042F8043B8A42D36133
:101AB000FAD103814381704738B50446202383F36C
:101AC0001188002500F10C0300F13002416043F859
:101AD000045B9342FBD1204601F048F802232370B7
:101AE00085F3118838BD000070B500EB8103054611
:101AF00050690E461446DA6018B110220021FFF733
:101B00005BFAA06918B110220021FFF755FA31469F
:101B10002846BDE8704001F03BB90000038900F1A0
:101B20003002002103F001030381438903F0010324
:101B3000438100F1100343F8041B9342FBD101F0F1
:101B4000BFB90000F0B4012500EB810447898D4046
:101B5000E4683D43A469458123600023A26063607B
:101B6000F0BC01F0DBB90000F0B4012500EB81040A
:101B700007898D40E4683D43646905812360002343
:101B8000A2606360F0BC01F053BA0000022300F1D0
:101B90000C0200F1300110B5037004460023A0F8D8
:101BA000883080F88A3080F88B300381438142F896
:101BB000043B8A42FBD184F87030204601F07CF867
:101BC00063681B6823B120460021BDE81040184718
:101BD00010BD00000278436880F88C2005221B6845
:101BE00002700BB10421184770470000436890F859
:101BF0008C201B6802700BB105211847704700004C
:101C000090F8703070B5044613B1002380F870303E
:101C100004F18002204601F077F963689B6863BB9A
:101C200094F8805015F0600615D194F8813005F0D5
:101C30007F0545EA032540F202339D4200F00E8104
:101C40005BD8022D00F0DC803FD8002D00F08780AB
:101C5000012D00F0CF800021204601F00DFC002175
:101C6000204601F0FDFB63681B6813B10621204686
:101C70009847062384F8703070BD204698470028A6
:101C8000CED094F8872094F8863043EA0223A26FDE
:101C9000934238BFA36794F98030A56F002B4FF0B3
:101CA000200380F2FD80002D00F0EC80092284F8F2
:101CB000702083F311880021A36F626F2046FFF725
:101CC00053FF002383F3118870BDB5F5817F00F0C9
:101CD000B180B5F5407F49D0B5F5807FBBD194F890
:101CE0008230012BB7D1B4F8883023F00203A4F876
:101CF00088306667A667E667C3E740F201639D42E6
:101D00001ED8B5F5C06F3BD2B5F5A06FA3D1B4F81E
:101D10008030B3F5A06F0ED194F88230204684F85D
:101D20008A3001F027F863681B6813B1012120464F
:101D300098470323237000236367A367E367A0E743
:101D4000B5F5106F32D040F602439D4252D0B5F542
:101D5000006F80D104F18B036367012324E004F159
:101D60008803E56763670223A3678AE794F88230F4
:101D7000012B7FF470AFB4F8883043F00203B6E76C
:101D800094F885202046616894F884304D6843EAD1
:101D9000022394F8831094F88220A84700283FF487
:101DA0005AAF436863670368A367A4E72378042BEB
:101DB00010D1202383F311882046FFF7AFFE86F36E
:101DC00011886368032184F88B601B6821700BB154
:101DD0002046984794F88230002BACD084F88B30A2
:101DE0000423237063681B68002BA4D002212046C3
:101DF0009847A0E7374B63670223A36700239DE75B
:101E000094F88410204611F0800F01F00F010ED0DD
:101E100001F06CF8012806D002287FF41CAF2E4B8D
:101E2000A067636767E72D4BA567636763E701F00A
:101E30004FF8EFE794F88230002B7FF40CAF94F862
:101E4000843013F00F013FF476AF1A06204602D516
:101E500001F02AFB6FE701F01BFB6CE794F882307E
:101E6000002B7FF4F8AE94F8843013F00F013FF4A8
:101E700062AF1B06204602D501F0FEFA5BE701F0D7
:101E8000EFFA58E7142284F8702083F311882B4668
:101E90002A4629462046FFF755FE85F3118870BD76
:101EA0005DB1152284F8702083F311880021A36F9F
:101EB000626F2046FFF746FE03E70B2284F870208E
:101EC00083F311882B462A4629462046FFF74CFE0D
:101ED000E3E700BF5C410008544100085841000896
:101EE00038B590F870300446152B29D8DFE803F098
:101EF0003E28282828283E28280B29392828282841
:101F0000282828283E3E90F8871090F88620836F76
:101F100042EA01229A4214D9C268128AB3FBF2F54E
:101F200002FB15356DB9202383F311882B462A4611
:101F30002946FFF719FE85F311880A2384F87030CB
:101F400038BD142384F87030202383F311880023D4
:101F500020461A461946FFF7F5FD002383F3118842
:101F600038BDC36F03B198470023E7E7002101F0B4
:101F700083FA0021204601F073FA63681B6813B1ED
:101F80000621204698470623D8E7000090F87020E5
:101F9000152A38B5044622D80123934040F6416201
:101FA00013421DD113F480150FD19B0217D50B23BB
:101FB00080F87030202383F311882B462A46294667
:101FC000FFF7D2FD85F3118838BDC3689B695B6854
:101FD0002BB9C36F03B19847002384F8703038BD24
:101FE000002101F049FA0021204601F039FA636826
:101FF0001B6813B10621204698470623EDE7000031
:10200000024B00221B605B609A607047AC2A002084
:10201000002382680374054B1B6899689142FBD2C8
:102020005A6803604260106058607047AC2A002014
:1020300008B5202383F31188037C032B05D0042BE0
:102040000DD02BB983F3118808BD436900221A60B3
:102050004FF0FF334361FFF7DBFF0023F2E790E827
:102060000C001A6002685360F2E7000000238268E7
:102070000374054B1B6899689142FBD85A6803604A
:102080004260106058607047AC2A0020054B196907
:1020900008741868026853601A6018610123037499
:1020A000FEF792B9AC2A00204B1C30B5054687B02C
:1020B0000A4C10D0236901A8094A00F0D3F8284639
:1020C000FFF7E4FF049B13B101A800F007F92369AF
:1020D000586907B030BDFFF7D9FFF8E7AC2A0020F8
:1020E0003120000838B50C4D044641612B698168E8
:1020F0009A68914203D8BDE83840FFF789BF184677
:10210000FFF786FF01232C61014623742046BDE8BA
:102110003840FEF759B900BFAC2A0020044B1A68BA
:102120001B6990689B68984294BF0020012070470B
:10213000AC2A002010B5084C236820691A68546046
:102140002260012223611A74FFF790FF0146206983
:10215000BDE81040FEF738B9AC2A002082600222A8
:1021600002740022427470478368A3F17C0243F832
:102170000C2C026943F83C2C426943F8382C074A7E
:1021800043F81C2CC268A3F1180043F8102C02225B
:1021900003F8082C002203F8072C7047E10300081D
:1021A00010B5202383F31188FFF7DEFF00210446DA
:1021B000FFF798FF002383F31188204610BD00002D
:1021C000024B1B6958610F20FFF760BFAC2A00204B
:1021D000202383F31188FFF7F3BF000008B5014601
:1021E000202383F311880820FFF75EFF002383F389
:1021F000118808BD49B1064B42681B6918605A60D6
:10220000136043600420FFF74FBF4FF0FF3070476B
:10221000AC2A00200368984206D01A680260506019
:1022200018465961FFF7F4BE7047000038B5044600
:102230000D462068844200D138BD036823605C608D
:102240004561FFF7E5FEF4E7054B03F114025A611F
:102250009A614FF0FF32DA6100221A62704700BFC4
:10226000AC2A0020F8B5036102291A4B0646C26069
:1022700038BF02215C6A184B1A461F4652F8145F99
:1022800095420AD1586198611C6205604560816081
:102290000819BDE8F84001F0E1BA186AAB68241AE1
:1022A0000C1902D3E41A2D6804E09C4202D22044A7
:1022B00001F0E4FAAB689C42F4D86B683560736057
:1022C0001E604FF0FF336E60B460A968091BA960FF
:1022D000FB61F8BD000C0040AC2A002010B41A4C81
:1022E000234653F8141F814210D0416802680A60E7
:1022F000026851609A424FF00001C16003D09368B8
:1023000081680B4493605DF8044B70470A680020B5
:102310009A4262615360C86003D15DF8044B01F0DA
:10232000A7BA936888680344206A9360074A526A90
:10233000121A9342E7D9991A5DF8044B012998BF04
:10234000931C184401F09ABAAC2A0020000C0040FB
:1023500000207047FEE70000704700004FF0FF309C
:1023600070470000022906D0032906D0012906483B
:1023700018BF0020704705487047032A9ABF0448D9
:1023800000EBC2000020704724420008D84100083A
:102390002424002070B59AB006460846144601ADC4
:1023A000294600F095F82846FEF7FEFDC0B2431C12
:1023B0005B0086E8180023700323023404F8013C14
:1023C00000231946DAB20234904201D81AB070BD27
:1023D000EA5C013304F8011C04F8022CF2E7000067
:1023E00008B5202383F311880348FFF7D3FA0023AD
:1023F00083F3118808BD00BFEC2A002010B5044605
:10240000052916D8DFE801F016150316161D20233E
:1024100083F311880E4A0121FFF766FB20460D4A1F
:102420000221FFF761FB0C48FFF77AFA002383F3E0
:10243000118810BD202383F311880748FFF746FA5F
:10244000F4E7202383F311880348FFF75DFAEDE7F3
:102450006041000884410008EC2A002038B50C4D8A
:102460000C4C2A460C4904F10800FFF793FF05F1D4
:10247000CA0204F110000949FFF78CFF05F5CA7282
:1024800004F118000649BDE83840FFF783BF00BFDC
:10249000B42F002024240020B0410008B4410008DB
:1024A000BF41000870B5044608460D46FEF77CFDA6
:1024B000C6B22046013403780BB9184670BD3246C7
:1024C0002946FEF75BFD0028F3D1012070BD000016
:1024D0002DE9F84F05460C46FEF766FD2A49C6B2BF
:1024E0002846FFF7DFFF08B10136F6B22749284634
:1024F000FFF7D8FF08B11036F6B2632E0DD8DFF81B
:102500008890DFF888A0224FDFF88CB0DFF88C804D
:102510002E7846B92670BDE8F88F29462046BDE8DA
:10252000F84F01F0BDBD252E2AD107224946284685
:10253000FEF724FD50B9D8F800300735083444F8C8
:10254000083CD8F8043044F8043CE1E7082251463E
:102550002846FEF713FD98B9A21C0E4B13F8011F75
:10256000023209095B45C95D02F8041C197801F0C3
:102570000F01C95D02F8031CF0D118340835C7E714
:10258000267001350134C3E744420008BF4100080A
:1025900055420008FFE7F11F0BE8F11F4C4200080D
:1025A000BFF34F8F044B1A695107FCD1D3F81021A8
:1025B0005207F8D1704700BF0020005208B50D4BFC
:1025C0001B78ABB9FFF7ECFF0B4BDA68D10704D5EA
:1025D0000A4A5A6002F188325A60D3F80C21D207B5
:1025E00006D5064AC3F8042102F18832C3F8042153
:1025F00008BD00BF123200200020005223016745B1
:1026000008B5114B1B78F3B9104B1A69510703D564
:10261000DA6842F04002DA60D3F81021520705D59B
:10262000D3F80C2142F04002C3F80C21FFF7B8FFA9
:10263000064BDA6842F00102DA60D3F80C2142F06E
:102640000102C3F80C2108BD123200200020005204
:102650000F289ABF00F580604004002070470000FA
:102660004FF4003070470000102070470F2808B565
:102670000BD8FFF7EDFF00F500330268013204D1FB
:1026800004308342F9D1012008BD002008BD0000BC
:102690000F2810B504463FD8FFF782FFFFF78EFFE3
:1026A0001E484FF0FF33072C4361C0F814311DD88A
:1026B0000361FFF775FF230243F02403C360C3687F
:1026C00043F08003C36003695A07FCD4FFF768FF37
:1026D0002046FFF7BDFF4FF4003100F0F7F8FFF799
:1026E0008FFF2046BDE81040FFF7C0BFC0F8103193
:1026F000FFF756FFA4F108031B0243F02403C0F8C0
:102700000C31D0F80C3143F08003C0F80C31D0F814
:1027100010315B07FBD4D9E7002010BD0020005228
:102720002DE9F84F40EA020305460E461746DB0640
:1027300056D13446DFF8C090DFF8C0A0FFF73EFF67
:102740003B1B33441F2B04D8FFF75AFF0120BDE881
:10275000F88F20222146284601F092FC002837D02D
:1027600005F17843214A22489342224B98BF98466C
:1027700003F5827392BFD346C8469B46A3F1080374
:1027800088BF1846FFF70CFF4FF0FF3304F11C0120
:10279000A5EB040ECBF80030036843F0020303609E
:1027A000231FD8F8002012F0050FFAD153F8042F98
:1027B00099424EF80320F4D1BFF34F8FFFF7F0FE9C
:1027C0004FF0FF33CBF80030036823F002030360BF
:1027D00020222146284601F053FC20B1FFF710FFCC
:1027E0000020BDE8F88F20352034A9E7FFFF0F0057
:1027F0000C200052102000521021005214200052D0
:1028000010B5084C237828B153B9FFF7D7FE012340
:10281000237010BD23B12070BDE81040FFF7F0BE5B
:1028200010BD00BF1232002002440439064BD2B260
:1028300010B5904200D110BD441C00B253F82000E6
:1028400041F8040FE0B2F4E7504000580F4B30B5A8
:102850001C6F240405D41C6F1C671C6F44F40044D7
:102860001C670B4C024404392368D2B243F48073D2
:102870002360084B904200D130BD441C51F8045FE6
:1028800000B243F82050E0B2F4E700BF0044025821
:10289000004802585040005807B5012201A9002005
:1028A000FFF7C2FF019803B05DF804FB13B50446BF
:1028B000FFF7F2FFA04206D002A90122002041F852
:1028C000044DFFF7C3FF02B010BD00000144BFF389
:1028D0004F8F064B884204D3BFF34F8FBFF36F8FE8
:1028E0007047C3F85C022030F4E700BF00ED00E061
:1028F000034B1B685B0142BF0122024B1A707047F9
:10290000D044025813320020014B1878704700BFA2
:1029100013320020064A536823F001035360EFF39B
:102920000983683383F30988002383F31188704790
:1029300030EF00E010B5202383F31188104B5B6863
:1029400013F4006318D0F1EE103AEFF309844FF05E
:10295000807344F84C3C0B4BDB6844F8083CA4F112
:10296000680383F30988FFF7D9FB18B1064B44F8D5
:10297000503C10BD054BFAE783F3118810BD00BF32
:1029800000ED00E030EF00E0F1030008F403000880
:10299000F0B5BFF34F8FBFF36F8F1D4B0021C3F80E
:1029A0005012BFF34F8FBFF36F8F5A6942F400325A
:1029B0005A61BFF34F8FBFF36F8FC3F88410BFF31B
:1029C0004F8FD3F8802043F6E076C2F3C904C2F3F8
:1029D0004E32A507520102EA060E284621464EEA6B
:1029E0000007013900F14040C3F860724F1CF6D176
:1029F000203A12F1200FEED1BFF34F8F5A6942F403
:102A000080325A61BFF34F8FBFF36F8FF0BD00BFAD
:102A100000ED00E0FEE70000084A094B09498B423F
:102A200004D3094A0021934205D3704752F8040F9A
:102A300043F8040BF3E743F8041BF4E740440008B1
:102A4000603500206035002060350020D0F89430DB
:102A5000002230B51146D0F890409D684FF0FF300D
:102A600004EB421301329542C3F80019C3F8101960
:102A7000C3F80809C3F8001BC3F8101BC3F8080B00
:102A8000EED24FF00113C4F81C3830BD00EB8103C7
:102A90002DE9F04FD3F80CE04F1C4FEA4118DEF857
:102AA00014403F03D4F800C06568D0F89020654515
:102AB0000AD30120D2F8343800FA01F123EA0101E7
:102AC000C2F83418BDE8F08FACEB0503BEF8106017
:102AD000B34228BF334602EB0806D6F81869B6B2EF
:102AE000B3EB860F13D8A6683A449946A6F1040AB8
:102AF0005AF804BFB9F1040FC2F800B002D9A9F125
:102B00000409F5E71E442B44A6606360CCE700206F
:102B1000BDE8F08F890141F02001016103699B0646
:102B2000FCD4122000F03ABF10B50A4C2046FEF744
:102B3000B3FF094BC4F89030084BC4F89430084CEC
:102B40002046FEF7A9FF074BC4F89030064BC4F8A7
:102B5000943010BD14320020000008408C42000860
:102B6000B032002000000440984200080378012B96
:102B700070B505465DD1494BD0F89040984259D187
:102B8000474B0E216520D3F8D82042F00062C3F8ED
:102B9000D820D3F8002142F00062C3F80021D3F816
:102BA0000021D3F8802042F00062C3F88020D3F8DF
:102BB000802022F00062C3F88020D3F88030FEF736
:102BC000E5FB384BE360384BC4F800380023D5F8F8
:102BD0009060C4F8003EC02323604FF40413A36345
:102BE0003369002BFCDA01230C20336100F0D6FEA0
:102BF0003369DB07FCD4122000F0D0FE3369002BD0
:102C0000FCDA00262846A660FFF720FF6B68C4F8B0
:102C10001068DB68C4F81468C4F81C68002B3AD14B
:102C2000224BA3614FF0FF336361A36843F00103BC
:102C3000A36070BD1E4B9842C8D1194B0E214D2088
:102C4000D3F8D82042F00072C3F8D820D3F800217E
:102C500042F00072C3F80021D3F80021D3F880209D
:102C600042F00072C3F88020D3F8802022F0007276
:102C7000C3F88020D3F88020D3F8D82022F08062D7
:102C8000C3F8D820D3F8002122F08062C3F80021D5
:102C9000D3F8003193E7074BC3E700BF143200209D
:102CA000004402584014004003002002003C30C0A1
:102CB000B0320020083C30C0F8B5D0F8904005464E
:102CC00000214FF000662046FFF724FFD5F894104E
:102CD00000234FF001128F684FF0FF30C4F83438F2
:102CE000C4F81C2804EB431201339F42C2F8006968
:102CF000C2F8006BC2F80809C2F8080BF2D20B68E0
:102D0000D5F89020C5F898306362102313611669D6
:102D100016F01006FBD1122000F040FED4F8003867
:102D200023F4FE63C4F80038A36943F4402343F05E
:102D30001003A3610923C4F81038C4F814380B4BEE
:102D4000EB604FF0C043C4F8103B094BC4F8003BA4
:102D5000C4F81069C4F80039D5F8983003F11002AE
:102D600043F48013C5F89820A362F8BD68420008B8
:102D700040800010D0F8902090F88A10D2F80038E7
:102D800023F4FE6343EA0113C2F8003870470000E1
:102D90002DE9F0410EB20D4600EB8608D8F80C1074
:102DA0000F6807F00303022B53D0032B53D03F4A85
:102DB0003F4F012B18BF1746D0F890404FEA451EF1
:102DC000002205F1100C04EB0E03C3F8102B8A69E6
:102DD000002A42D04A8A05F158033A435B01E25087
:102DE0000123D4F81C2803FA0CF31343C4F81C384D
:102DF000A64400234A69CEF8103905F13F03002AA2
:102E00003BD00A8A04EB8303898B9208012988BF8F
:102E10004A43D0F89810561841EA02422946C0F8B1
:102E2000986020465A60FFF775FED8F80C301B8A70
:102E300043EA85531F4305F148035B01E750012333
:102E4000D4F81C2803FA05F51543C4F81C58BDE84E
:102E5000F081184FB0E7184FAEE704EB4613D3F8F4
:102E6000002B22F40042C3F8002B0123D4F81C28C5
:102E700003FA0CF322EA0303B8E704EB83030F4AD7
:102E800004EB461629465A602046FFF743FED6F863
:102E90000039012223F4004302FA05F5C6F800398F
:102EA000D4F81C3823EA0505CFE700BF00800010E6
:102EB000008004100080081000800C100004000244
:102EC000D0F894201268C0F89820FFF7BFBD00002A
:102ED0005831D0F8903049015B5813F4004004D0C9
:102EE00013F4001F14BF0120022070474831D0F8AE
:102EF000903049015B5813F4004004D013F4001FD4
:102F000014BF01200220704700EB8101CB68196AD1
:102F10000B6813604B6853607047000000EB81033F
:102F200030B5DD68AA691368D36019B9402B84BF36
:102F3000402313606B8A1468D0F890201C4402EB85
:102F40004110013C09B2B4FBF3F46343033323F0B3
:102F5000030343EAC44343F0C043C0F8103B2B686B
:102F600003F00303012B0ED1D2F8083802EB411015
:102F700013F4807FD0F8003B14BF43F0805343F03C
:102F80000053C0F8003B02EB4112D2F8003B43F083
:102F90000443C2F8003B30BD2DE9F041D0F8906009
:102FA00005460C4606EB4113D3F8087B3A07C3F8F5
:102FB000087B08D5D6F814381B0704D500EB81032D
:102FC000DB685B689847FA072FD5D6F81438DB071B
:102FD0002BD505EB8403D968CCB98B69488A5E6828
:102FE000B6FBF0F200FB12628AB91868DA68904208
:102FF0000DD2121A83E81400202383F3118821468E
:103000002846FFF78BFF84F31188BDE8F081012388
:1030100003FA04F26B8923EA02036B81CB6823B1C4
:1030200021462846BDE8F0411847BDE8F081000080
:1030300000EB81034A0170B5DD68D0F890306C690F
:103040002668E66056BB1A444FF40020C2F8100907
:103050002A6802F00302012A0AB20ED1D3F8080846
:1030600003EB421410F4807FD4F8000914BF40F041
:10307000805040F00050C4F8000903EB4212D2F82F
:10308000000940F00440C2F800090122D3F83408D6
:1030900002FA01F10143C3F8341870BD19B9402E8A
:1030A00084BF4020206020681A442E8A841940F092
:1030B0000050013CB4FBF6F440EAC440C6E700000F
:1030C0002DE9F041D0F8906004460D4606EB41131F
:1030D000D3F80879C3F80879FB071CD5D6F810385F
:1030E000DA0718D500EB8103D3F80CE0DEF81430D2
:1030F000D3F800C0DA6894451BD2A2EB0C024FF063
:1031000000081A60C3F80480202383F31188FFF7B6
:103110008FFF88F311883B0618D50123D6F8342891
:10312000AB40134212D029462046BDE8F041FFF7DC
:10313000ADBC012303FA01F2038923EA02030381F0
:10314000DEF80830002BE6D09847E4E7BDE8F081D0
:103150002DE9F047D0F8905004466E69AB691E40E7
:10316000F1046E6103D5BDE8F047FEF70FBD002EF8
:1031700012DAD5F8003E9A0705D0D5F8003E23F0C4
:103180000303C5F8003ED5F80438204623F00103B8
:10319000C5F80438FEF72AFD330502D52046FEF7B0
:1031A00019FDB7040CD5D5F8083813F0060FEB68F5
:1031B00023F470530CBF43F4105343F4A053EB605B
:1031C000300704D56368DB680BB120469847F102ED
:1031D00000F1A180B2020BD5D4F8908000274FF007
:1031E0000109D4F89430F9B29B688B4280F0D28008
:1031F000F3061AD5D4F890100A6AC2F30A1702F03F
:103200000F0302F4F012B2F5802F00F0EB80B2F55C
:10321000402F0AD104EB830301F58051DB68186A63
:1032200000231A469F4240F0D1803003D5F8185849
:1032300035D5E90303D500212046FFF7ADFEAA03EB
:1032400003D501212046FFF7A7FE6B0303D502211A
:103250002046FFF7A1FE2F0303D503212046FFF7E9
:103260009BFEE80203D504212046FFF795FEA90244
:1032700003D505212046FFF78FFE6A0203D50621FC
:103280002046FFF789FE2B0203D507212046FFF7D2
:1032900083FEEF0103D508212046FFF77DFE700372
:1032A00040F1C780E90703D500212046FFF708FF5A
:1032B000AA0703D501212046FFF702FF6B0703D5BC
:1032C00002212046FFF7FCFE2F0703D503212046ED
:1032D000FFF7F6FEEE0603D504212046FFF7F0FEC9
:1032E000A80603D505212046FFF7EAFE690603D5A7
:1032F00006212046FFF7E4FE2A0603D507212046D3
:10330000FFF7DEFEEB0540F1948020460821BDE882
:10331000F047FFF7D5BED4F890904FF000084FF07B
:10332000010AD4F894305FFA88F79B68BB42FFF437
:1033300051AF09EB4713D3F8002902F44022B2F54C
:10334000802F24D1D3F80029002A20DAD3F80029CD
:1033500042F09042C3F80029D3F80029002AFBDB91
:103360003946D4F89000FFF7D5FB22890AFA07F313
:1033700022EA0303238104EB8703DB689B6813B114
:1033800039462046984739462046FFF77FFB08F12B
:103390000108C6E708EB4112D2F8003B03F44023D2
:1033A000B3F5802F10D1D2F8003B002B0CDA6289E4
:1033B00009FA01F322EA0303638104EB8103DB686A
:1033C000DB680BB12046984701370AE713F0030F7B
:1033D00000D10A68072B03F101039EBF0270120A95
:1033E00001301FE704EB830301F58051DA6890692F
:1033F0000268D0F808C04068A2EB000E0022104618
:10340000974208D1DB689B699A683A449A605A6887
:1034100017445F6009E712F0030F00D10868964572
:1034200002F1010282BF8CF80000000A0CF1010CCD
:10343000E6E7BDE8F087000008B50348FFF788FE1F
:10344000BDE80840FFF776BA1432002008B50348FB
:10345000FFF77EFEBDE80840FFF76CBAB0320020EF
:10346000D0F8903003EB4111D1F8003B43F4001346
:10347000C1F8003B70470000D0F8903003EB4111D9
:10348000D1F8003943F40013C1F800397047000047
:10349000D0F8903003EB4111D1F8003B23F4001336
:1034A000C1F8003B70470000D0F8903003EB4111A9
:1034B000D1F8003923F40013C1F800397047000037
:1034C00030B50433039C0172002104FB0325C36162
:1034D000049B00600363059B4060C1604261026120
:1034E0008561046242628162C162436330BD000053
:1034F0000022416AC260416101616FF00101826294
:10350000C262FEF793BE000003694269934203D191
:10351000C2680AB100207047181D7047036919601E
:103520000021C2680132C260C269134482699342B9
:10353000036124BF436A0361FEF76CBE38B50446DD
:103540000D46E3683BB162690020131D1268A36257
:103550001344E36238BD237A33B929462046FEF787
:1035600049FE0028EDDA38BD6FF00100FBE70000EE
:10357000C368C269013BC3604369134482699342D3
:10358000436124BF436A436100238362036B03B139
:103590001847704770B52023044683F31188866A64
:1035A0003EB9FFF7CBFF054618B186F311882846D0
:1035B00070BDA36AE26A13F8015B9342A36202D36F
:1035C0002046FFF7D5FF002383F31188EFE70000C3
:1035D0002DE9F84F04460E4690469946202787F37A
:1035E00011880025AA46D4F828B0BBF1000F09D1F4
:1035F00049462046FFF7A2FF20B18BF311882846E9
:10360000BDE8F88FA16AA8EB050BE36A5B1A9B453E
:1036100028BF9B46BBF1400F1BD9334601F1400246
:1036200051F8040B914243F8040BF9D1A36A4036D8
:1036300040354033A362A26AE36A9A4202D320462D
:10364000FFF796FF8AF311884545D8D287F3118892
:10365000C9E730465A46FDF787FCA36A5E445D44DD
:103660005B44A362E7E7000010B5029C04330172DB
:10367000C36103FB0421002300608362C362039BD8
:1036800040600363049BC460426102618161046223
:103690004262436310BD0000026A6FF00101C26024
:1036A000426A4261026100228262C262FEF7BEBDCE
:1036B000436902699A4203D1C2680AB10020704787
:1036C000184650F8043B0B6070470000C3680021A7
:1036D000C2690133C3604369134482699342436101
:1036E00024BF436A4361FEF795BD000038B5044628
:1036F0000D46E3683BB1236900201A1DA262E2690E
:103700001344E36238BD237A33B929462046FEF7D5
:1037100071FD0028EDDA38BD6FF00100FBE7000015
:1037200003691960C268013AC260C26913448269C0
:103730009342036124BF436A036100238362036BE6
:1037400003B118477047000070B5202304460E46A9
:1037500083F31188856A35B91146FFF7C7FF10B1A9
:1037600085F3118870BDA36A1E70A36AE26A0133F3
:103770009342A36204D3E16920460439FFF7D0FFE6
:10378000002080F3118870BD2DE9F84F04460D46E6
:1037900091469A464FF0200888F311880026B346D8
:1037A000A76A4FB951462046FFF7A0FF20B187F323
:1037B00011883046BDE8F88FA06AA9EB0603E76AD6
:1037C0003F1A9F4228BF1F46402F1BD905F14003D7
:1037D00055F8042B9D4240F8042BF9D1A36A4036DA
:1037E0004033A362A26AE36A9A4204D3E1692046A5
:1037F0000439FFF795FF8BF311884E45D9D288F332
:103800001188CDE729463A46FDF7AEFBA36A3D4451
:103810003E443B44A362E5E7026943699A4203D10F
:10382000C3681BB9184670470023FBE7836A002B67
:10383000F8D0043B9B1AF5D01360C368013BC3600A
:10384000C3691A4483699A42026124BF436A0361CF
:10385000002383620123E5E700F050B9034B002207
:1038600058631A610222DA60704700BF000C004002
:103870000022014BDA607047000C0040014B586396
:10388000704700BF000C0040FEE7000010B5194C67
:10389000FEF7B6FBFEF7D8FC802217492046FEF75C
:1038A0005DFC012344F8180C0374144B144AD968C6
:1038B00021F4E0610904090C0A431249DA60CA687C
:1038C00042F08072CA60104A1049C2F8B01F1168F5
:1038D00041F0010111601022DA77202283F82220C2
:1038E000002383F3118862B60948BDE81040FEF753
:1038F00057BC00BFD42A0020A442000800ED00E01D
:103900000003FA05F0ED00E0001000E055CEACC574
:10391000AC4200082DE9F84F1E4C4FF00008DFF8CC
:103920007890656904F11407D9F82430266AAA68EA
:103930009E1B96421CD34FF0200AAA68236AD5F832
:103940000CB0B61A134423622B68BB425F606361FC
:10395000C5F80C8001D1FFF78BFF88F31188286927
:10396000D8478AF311886569AB689E42E5D2DBE7E8
:103970006269BA420CD0916823628E1B9660A86877
:1039800002282CBF1818981CBDE8F84FFFF776BF27
:10399000BDE8F88FAC2A0020000C0040034B5968AA
:1039A0005A68521A9042FBD8704700BF001000E0DE
:1039B0004B6843608B688360CB68C3600B6943616D
:1039C0004B6903628B6943620B68036070470000B8
:1039D00008B52C4B40F2FF712B48D3F888200A43DE
:1039E000C3F88820D3F8882022F4FF6222F007026F
:1039F000C3F88820D3F88820D3F8E0200A43C3F81E
:103A0000E020D3F808210A43C3F808211F4AD3F85D
:103A100008311146FFF7CCFF1D4802F11C01FFF7EA
:103A2000C7FF1C4802F13801FFF7C2FF1A4802F134
:103A30005401FFF7BDFF194802F17001FFF7B8FF0D
:103A4000174802F18C01FFF7B3FF164802F1A801F5
:103A5000FFF7AEFF144802F1C401FFF7A9FF1348B6
:103A600002F1E001FFF7A4FF114802F1FC01FFF7AA
:103A70009FFF104802F58C71FFF79AFFBDE80840E0
:103A800000F016B90044025800000258CC42000869
:103A90000004025800080258000C02580010025896
:103AA0000014025800180258001C02580020025846
:103AB000002402580028025808B500F0CFFAFFF79A
:103AC000E5FEFEF715FFBDE80840FEF7C7BC0000A5
:103AD00070470000084B1A69920710B508D50024FA
:103AE0001C61202383F31188FFF714FF84F31188EE
:103AF000BDE81040FEF71EBF000C0040124B08212D
:103B00003220D3F8E82042F00802C3F8E820D3F8C6
:103B1000102142F00802C3F810210C4AD3F81031EA
:103B2000D36B43F00803D363C722094B9A624FF06B
:103B3000FF32DA6200229A615A63DA605A60012227
:103B40005A611A60FDF722BC004402580010005C64
:103B5000000C0040F8B5514B0024D3F880204FF002
:103B6000FF32C3F88020D3F88010C3F88040D3F828
:103B70008010D3F88410C3F88420D3F88410C3F8DD
:103B80008440D3F88410D96F41F0FF4141F4FF0124
:103B900041F4DF4141F07F01D967D96F21F0FF4146
:103BA00021F4FF0121F4DF4121F07F01D967D96FB2
:103BB000D3F888106FEA41516FEA5151C3F8881069
:103BC000D3F88810C1F30A01C3F88810D3F888101D
:103BD000D3F89010C3F89020D3F89010C3F8904019
:103BE000D3F89010D3F89410C3F89420D3F894101D
:103BF000C3F89440D3F89410D3F89810C3F89820E1
:103C0000D3F89810C3F89840D3F89810D3F88C10D4
:103C1000C3F88C20D3F88C10C3F88C40D3F88C10E8
:103C2000D3F89C10C3F89C20D3F89C20C3F89C4088
:103C3000D3F89C3000F0F2F9194B07229A60194A28
:103C4000DA60194A1A6105225A60184A536A43F425
:103C500080335362C2F88440BFF34F8FD2F8803074
:103C600043F6E076C3F3C904C3F34E33A5075B0103
:103C700003EA060E284621464EEA0007013900F104
:103C80004040C2F874724F1CF6D1203B13F1200F54
:103C9000EED1BFF34F8FBFF36F8FF8BD00440258D2
:103CA00090ED00E0000004301B00080300ED00E090
:103CB00001225E4B5E491A605E4B19609A605E4A53
:103CC000DA6000221A614FF440429A619A699204C4
:103CD000FCD51A6842F480721A60584B1A6F12F4BD
:103CE000407F04D04FF480321A6700221A671A68A6
:103CF00042F001021A60514A134611684807FCD588
:103D0000002111611A6912F03802FBD101211960FA
:103D10004FF0804159605A67494ADA62494A1A614C
:103D20001A6842F480321A60444A134611688903C3
:103D3000FCD5116841F0800111601A68D205FCD5EC
:103D4000414A42499A6200225A631963A1F5C0218F
:103D5000DA63A1F50D7199635A643D4A1A643D4ACC
:103D6000DA621A6842F0A8521A60344B1A6802F0FC
:103D70002852B2F1285FF9D1482222219A614FF4EA
:103D80008862DA6140221A624FF00052DA64324AE5
:103D90001A65324A5A6502F1726202F571429A65F9
:103DA0002F4A11601A6942F003021A61234B1A6903
:103DB00002F03802182AFAD1D3F8DC2042F000527F
:103DC000C3F8DC20D3F8042142F00052C3F80421E8
:103DD000D3F80421D3F8DC2042F08042C3F8DC2081
:103DE000D3F8042142F08042C3F80421D3F804211F
:103DF000D3F8DC2042F00042C3F8DC20D3F80421E1
:103E000042F00042C3F80421D3F80421D3F8F4208F
:103E100042F00202C3F8F420D3F81C2142F002025F
:103E2000C3F81C21D3F81C31704700BF0881005132
:103E300000C000F00048025802000001004402588F
:103E40000000FF0100889008222050003F02070177
:103E50002F040407FD0BFF01000001100010E0001B
:103E600000200052084A08B5936811680B4003F01F
:103E70000103936023B1054A13680BB1506898475A
:103E8000BDE80840FEF756BD80000058C025002060
:103E9000084A08B5936811680B4003F00203936069
:103EA00023B1054A93680BB1D0689847BDE8084034
:103EB000FEF740BD80000058C0250020084A08B524
:103EC000936811680B4003F00403936023B1054A23
:103ED00013690BB150699847BDE80840FEF72ABD49
:103EE00080000058C0250020084A08B59368116872
:103EF0000B4003F00803936023B1054A93690BB1AB
:103F0000D0699847BDE80840FEF714BD800000580E
:103F1000C0250020084A08B5936811680B4003F0DB
:103F20001003936023B1054A136A0BB1506A984796
:103F3000BDE80840FEF7FEBC80000058C025002008
:103F4000174B10B59C681A68144004F478729A6094
:103F5000A30604D5134A936A0BB1D06A984760064A
:103F600004D5104A136B0BB1506B9847210604D54A
:103F70000C4A936B0BB1D06B9847E20504D5094A04
:103F8000136C0BB1506C9847A30504D5054A936C8C
:103F90000BB1D06C9847BDE81040FEF7CBBC00BF1A
:103FA00080000058C02500201A4B10B59C681A6884
:103FB000144004F47C429A60620504D5164A136DDD
:103FC0000BB1506D9847230504D5134A936D0BB17F
:103FD000D06D9847E00404D50F4A136E0BB1506EB4
:103FE0009847A10404D50C4A936E0BB1D06E984744
:103FF000620404D5084A136F0BB1506F984723042D
:1040000004D5054A936F0BB1D06F9847BDE81040B7
:10401000FEF790BC80000058C0250020062108B59E
:104020000846FDF7B3F906210720FDF7AFF9062191
:104030000820FDF7ABF906210920FDF7A7F90621B5
:104040000A20FDF7A3F906211720FDF79FF90621A5
:104050002820BDE80840FDF799B9000008B5FFF732
:1040600079FDFDF769F8FDF73BFBFDF713FDFDF763
:10407000E5FBFFF72DFDBDE80840FFF7EDBB0000B5
:1040800010B501390244904201D1002010BD10F852
:10409000013B11F8014FA342F5D0181B10BD0000E1
:1040A000034611F8012B03F8012B002AF9D17047C0
:1040B000121012131211000001105A0003105900BF
:1040C0000120580003205600EC2A00204026002042
:1040D00053544D333248373F3F3F0053544D3332F2
:1040E000483734332F373533000000000096000086
:1040F00000000000000000000000000000000000C0
:104100000000000000000000A91600089516000835
:10411000D1160008BD160008C9160008B51600081B
:10412000A11600088D160008DD160008000000002A
:10413000B5170008A1170008DD170008C917000807
:10414000D5170008C1170008AD1700089917000817
:104150003918000800000000010000000000000005
:104160000200000000000000E11900084D1A0008DC
:1041700040004000842F0020942F00200200000007
:10418000000000000300000000000000911A000879
:104190000000000010000000A42F0020000000001C
:1041A00001000000000000001432002001010200A4
:1041B0006D526F0025424F415244252D424C00253F
:1041C00053455249414C2500FD2300086523000852
:1041D0004D190008E123000843000000E0410008F9
:1041E00009024300020100C032090400000102027A
:1041F000010005240010010524010001042402022D
:104200000524060001070582030800FF09040100D8
:10421000020A0000000705010240000007058102B4
:1042200040000000120000002C42000812011001A2
:104230000200004009124157000201020301000080
:104240000403090425424F41524425006D526F4E2C
:10425000657875730030313233343536373839414B
:10426000424344454600000000000000011C0008D5
:10427000E11E00088D1F0008400040004C33002064
:104280004C330020010000005C330020800000005F
:1042900040010000080000000001000000040000D0
:1042A000080000006D61696E00000000C442000853
:1042B00068330020603500200100000089380008C4
:1042C0000000000069646C65000000000050806A16
:1042D00000000000AAAAAAAA00000040FFFF0000F8
:1042E0000000000000A00A000500400100000000DE
:1042F000AAAAAAAA00004001FDFF000000000000D9
:10430000000000000000000000000000AAAAAAAA05
:1043100000000000FFFF000000000000000000009F
:104320000000000000000000AAAAAAAA00000000E5
:10433000FFFF0000000000000000000040810200BC
:1043400000000000AAAAAAAA40410100FFFF000045
:1043500000000070070000000000000000000000E6
:10436000AAAAAAAA00000000FFFF000000000000A7
:10437000000000000000000000000000AAAAAAAA95
:1043800000000000FFFF000000000000000000002F
:104390000000000000000000AAAAAAAA0000000075
:1043A000FFFF00000000000000000000000000000F
:1043B00000000000AAAAAAAA00000000FFFF000057
:1043C00000000000000000000000000000000000ED
:1043D000AAAAAAAA00000000FFFF00000000000037
:1043E000000000000000000000000000AAAAAAAA25
:1043F00000000000FFFF00000000000000000000BF
:10440000FF00000000000000D04000083F00000056
:1044100050040000DB4000083F0000000096000050
:1044200000000800040000004042000800000000F6
:10443000000000000000000000000000000000007C
:044440000000000078
:00000001FF
